:10000000BA298207B234B234B234B234B134AE3425
:10001000AB34A834A734A534A334A234A0349F341D
:100020009E349D349B349A34993498349834973460
:100030009634953494349334933492349134903488
:1000400090348F348F348E348D348D348C348C34A2
:100050008B348B348A3489348934883488348734B7
:1000600087348634863485348534843484348334C8
:1000700083348234823482348134813400340034D5
:1000800001340134013402340234023403340334C1
:100090000434043404340534053406340634063498
:1000A0000734073407340834083409340934093470
:1000B0000A340A340A340B340B340C340C340C3448
:1000C0000D340D340D340E340E340E340F340F3421
:1000D0000F341034103410341134113411341234FC
:1000E00012341234133413341434143414341534D5
:1000F00015341534163416341634173417341734AF
:10010000183418341934193419341A341A341A3486
:100110001B341B341B341C341C341C341D341D3460
:100120001E341E341F341F341F3420342034213435
:10013000213421342234223422342334233423340E
:1001400024342434253425342634263426342734E4
:10015000283428342834293429342A342A342A34B7
:100160002B342B342C342D342D342E342E342E3489
:100170002F342F3430343034313432343234333459
:100180003334343434343534353436343734373426
:1001900038343834393439343A343B343C343D34EF
:1001A0003D343E343E343F344034413442344234B2
:1001B000433444344534463447344834493449346C
:1001C0004A344C344D344E34503451345234533418
:1001D00055345634573459345B345C345E346034AF
:1001E0006234643469346B346E347034733478340C
:0601F0007D347D347E34F5
:100200008207543465346D34703441346C346D3449
:1002100032342034563432342E34313480344D3438
:100220002E344334733465346C34653420343934BB
:1002300039342F343034393480345F3454346534B5
:100240006D3470343D3480344D3469346E34203430
:1002500054343D3480344D34613478342034543453
:100260003D3480344834693420344C3469346D343E
:100270003D3480344C346F3420344C3469346D3424
:100280003D34803453346534743420344C346F340A
:10029000773420344C3469346D34693474348034A8
:1002A00053346534743420344834693467346834E2
:1002B00020344C3469346D346934743480344334BC
:1002C0006C3465346134723420344D3469346E34A6
:1002D0002F344D34613478343F34803450347234A8
:1002E00065347334733420342B34203474346F34D5
:1002F000203443346C347234803441346C3461348F
:1003000072346D3420344F346E342F344F346634AD
:1003100066343F348034503472346534733473340B
:1003200020342B34203466346F34723420344F340C
:100330004E34203480345034723465347334733422
:1003400020342B34203466346F34723420344F34EC
:1003500046344634803441346C34613472346D3404
:100360002034443469347334613462346C34653419
:1003700064348034860140308316860083128601FF
:1003800085010130831685008312043085008616AE
:10039000CE2386127F230130D82299230F30D82212
:1003A0001030AE00C223AE0BD22901306523A90064
:1003B00002306523A80004306523AA0003306523BA
:1003C000AB0005306523A70094019023E4222B089D
:1003D0002D02031CF0292D08AB00AE0003306B2367
:1003E0002A082D020318F9292D08AA00AE000430AE
:1003F0006B2380309000A0231D30D8222D08FC22D2
:100400008F309000A0235F309000B3239410290810
:100410002D0203180F2A28082D020318102A9414FD
:100420009418142A8511152A8515C0309000A02330
:100430002430D8222A08FC223E22C0309000A0237B
:100440002B30D8222B08FC223E22C0309000A02363
:100450003230D8222908FC223E22C0309000A0234E
:100460003A30D8222808FC223E22A718E529C030BD
:100470009000A023AB30D8223E22E529A71C422AB7
:10048000941886160830AE00AE0B482A8612080073
:10049000C2234E22A60026187422442A6122A600F6
:1004A000A61F542A0030080093006122A600A61F50
:1004B000552A130808006122A600A61F0800003074
:1004C0000800860180300614061B013006108614D1
:1004D000061B023086100615061B04300611861511
:1004E000061B08308611080090235030D822C030F7
:1004F0009000A0233230D8222908FC225B22A600DB
:100500002618882AA618A90A2619A903C823772A13
:1005100090234230D822C0309000A0233A30D82215
:100520002808FC225B22A60026189C2AA618A80AE6
:100530002619A803C8238B2A90235F30D822C03005
:100540009000A0236E30D8224E22A6002618B52A8D
:10055000A618AC2AC8239F2AE4222D08AB00AA00C3
:10056000AE0004306B2303306B2390237D30D82200
:10057000C0309000A023A71CC02A9B30D822C22ADA
:100580008B30D8224E22A6002618CA2AA618A70900
:10059000C823B82AC8232908AE0001306B232808D5
:1005A000AE0002306B232708AE0005306B23080035
:1005B0009500950301308A00150800219000901BDA
:1005C0000800B323950ADA2AAD0105110830AC0002
:1005D000851400008510851400008510031005188F
:1005E0000314AD0DAC0BEB2A0515F8302D02031CDE
:1005F0000800F830AD0008008A0101209A0096003A
:1006000017109A1F092B2D309000B3239A1317143B
:1006100096139901D7231C080F390319122B303E6A
:100620009000B3231D0E0F39303E9000B3231D08F8
:100630000F39303E9000B32343309000B3232F3066
:100640009000B3231D30980099019A0108309E0054
:1006500016080310980C03189907990C9A0C9E0B16
:100660002A2B04309E000310990C9A0C9E0B332BFE
:10067000171C3D2B9A099A0A990920309A070318EA
:10068000990A991F492B2D309000B32399019A099B
:100690009A0AD7231C080F390319512B303E9000BA
:1006A000B3231D0E0F39303E9000B3231D080F39C0
:1006B000303E9000B32346309000B32320309000AA
:1006C000B32320309000B323080089008316081458
:1006D00083120808080089002E0888000B08AE0065
:1006E0008B138316081555308900AA3089008814A9
:1006F0008818782B081183122E088B0008003330DD
:100700009000A02332309000A02328309000A02336
:100710000C309000A02306309000A0239023080006
:1007200001309000A02302309000A023CE23CE23DE
:100730000800C0309000A023CE23CE23CE23080093
:10074000100E0F3986008617CE23CE238613CE23B4
:10075000CE2310080F3986008617CE23CE238613AA
:10076000CE23CE230800100E0F39860006168617FA
:10077000861310080F398600061686178613CE23B7
:10078000CE230800FF309200CE23920BC42B08002A
:1007900033309200CE23920BCA2B0800FA3091001E
:1007A000910BD02BFA309100910BD42B0800031041
:1007B00010309E009B019C019D019A0D990D9D0D8D
:1007C0009C0D9B0D9E0BE52B00341D308400EF2308
:1007D0001C308400EF231B308400EF23DD2B03301B
:1007E00000079F009F198000303000079F009F1B6B
:0407F0008000003451
:00000001FF
